:020000040000FA
:06000000703002303A28C6
:08000800A000030EA100831209
:100010008B1C32288B1031181428B11C3228643004
:10002000010203183128182800001628172818285C
:1000300019281A281B281C281D281E281F283110A3
:10004000B114A810031005190314AA0DA90DA80DC9
:10005000B00B322831152A08AF002908AE00280855
:10006000AD00B11081010B11210E8300A00E200EF6
:02007000090085
:0C007400203084008001840A80300402E7
:10008000031C3C281230B0005E2183160C3085051D
:1000900087018312850187010730990000309A009B
:1000A000103083168E008312603083168F00831207
:1000B0000030831691009F008312C83083168100A0
:1000C000831231309000003083168C008312103080
:1000D0008B00A22181018E018F010B118B100B105F
:1000E0008C018B178220311998204021B30B802876
:1000F000031085190314B90DF03039020319E920F2
:10010000A52172286400311808000B1D08000B118E
:10011000B11031141230B000051D9328321483162B
:10012000011383120800321083160117831208008E
:1001300031110130B7008B132030370783169B0035
:100140001C141A088312A400A500C030A5061030A4
:10015000370783169B001C141A088312A300003073
:10016000370783169B001C141A088312A2008B17F2
:10017000321CC02822090339A200A309A409A50939
:1001800022082D02031DE32823082E02031DE32865
:1001900024082F02031DD52801303702031DD5285E
:1001A0003D18D5283D143E147B2125082F02031D40
:1001B000E32801303702031DE2283D1CE2283D10F0
:1001C0003E149F21E328B70A0230370203180800C3
:1001D0009B280130B600B300B400B500B70085011C
:1001E0008701B1138220B30B0F2903108519031463
:1001F000B90DF030390203193629B41F8501B41F37
:100200008701B40B0F293708B6080319B600031984
:100210000D29FF3085008700B6039630B400311DEC
:10022000F2283111321C19292D090339AD00AE090C
:10023000AF092F1CB1132F1CF228B11BF2282E1866
:10024000F228B1178B1320303707BB002F08BA00F4
:10025000492110303707BB002E08BA004921003071
:100260003707BB002D08BA0049218B17850187018C
:10027000B70AB60102303702031CF228A221080097
:100280003E1C08003E101030BB003D08BA0049215A
:1002900008008B133A0883161C159A0083123B083A
:1002A00083169B0055309D00AA309D009C1464006D
:1002B0009C1857291C1183128B17080083161030C5
:1002C0009B001C141A088312BD00831620309B006B
:1002D0001C141A088312DF00FF30D5000230D6004C
:1002E0000C30D700BA30D8003730D900DA30DA0015
:1002F0006F30DB0008000130BD000430C200C500D3
:100300000530C400C600CA000730C100C300C700E2
:10031000C800C9005F19C1175F19C2175F19C31759
:10032000DF19C4175F1AC5175F1AC6175F1AC717F8
:100330005F1AC8175F1BC917DF18CA1708008501A5
:10034000870108003D187B21080001303D05031995
:1003500008005F19AD295C1805165F19B129DC1872
:1003600085165F19B5295C190514DF19B929DC193F
:1003700085145F1ABD295C1A87145F1AC129DC1A1B
:1003800007155F1AC5295C1B07145F1AC929DC1BF6
:1003900087165F1BCD295D180716DF18D129DD18D8
:1003A0008715E6300E02031CE9295F1D05165F1D47
:1003B00085165F1D0514DF1D85145F1E87145F1EE3
:1003C00007155F1E07145F1E87165F1F0716DF1CC9
:1003D00087158F08031908008F01850187015508CB
:1003E000DE00E723D5005608DE00E723D6005708D5
:1003F000DE00551CE723D7005808DE00D51CE72394
:10040000D8005908DE00551DE723D9005A08DE0040
:10041000D51DE723DA005B08DE00551EE723DB006D
:100420005F1D2C2AC11B272AC11C0512C11C1B2AB7
:10043000051258190516CB0B3D2A5608CB00C101F1
:10044000D51BC114D81BC1105818C1103D2A051264
:10045000CB0B3D2AC1033D2AC10803190516031918
:100460003D2ACB0B3D2AD51BC1035508CB00D5181F
:100470005C14D51E5C10D51D5C105F1D592AC21B73
:10048000542AC21C8512C21C482A85125818851687
:10049000CC0B6A2A5608CC00C201D61BC2145A18CB
:1004A000C210D619C2106A2A8512CC0B6A2AC2035E
:1004B0006A2AC2080319851603196A2ACC0B6A2A0C
:1004C000D61BC2035608CC00D61ADC14561DDC100D
:1004D000561FDC105F1D862AC31B812AC31C051012
:1004E000C31C752A05105A190514CD0B972A5708F5
:1004F000CD00C301D71BC314D51AC310D719C3101D
:10050000972A0510CD0B972AC303972AC30803190E
:1005100005140319972ACD0B972AD71BC303570835
:10052000CD00571A5C15571F5C11D71D5C11DF1DDC
:10053000B32AC41BAE2AC41C8510C41CA22A851071
:10054000D51B8514CE0BCF2A5808CE00C401D81B6A
:10055000C414D71AC410D819C410CF2A8510CE0BD2
:10056000CF2AC403CF2ADF1FBE2ACE0BCF2A5808BA
:10057000CE00D51BDC15DA1FDC11CF2AC408031905
:1005800085140319CF2ACE0BCF2AD81BC4035808D1
:10059000CE00581ADC15D81FDC11D81DDC115F1EE7
:1005A000EB2AC51BE62AC51C8710C51CDA2A871052
:1005B000D51A8714CF0BFC2A5908CF00C501D91BC7
:1005C000C514561AC510D81BC510FC2A8710CF0BAE
:1005D000FC2AC503FC2AC508031987140319FC2A41
:1005E000CF0BFC2AD91BC5035908CF00D91B5C16B9
:1005F000D91F5C12D91C5C125F1E182BC61B132B53
:10060000C61C0711C61C072B0711D71A0715D00BDC
:10061000292B5A08D000C601DA1BC614D51AC610F9
:10062000D619C610292B0711D00B292BC603292B4D
:10063000C608031907150319292BD00B292BDA1B20
:10064000C6035A08D0005A1ADC165A1EDC12DA1FEA
:10065000DC125F1E452BC71B402BC71C0710C71C95
:10066000342B071059190714D10B562B5B08D100F6
:10067000C701DB1BC714D719C710DB19C710562BCE
:100680000710D10B562BC703562BC70803190714A5
:100690000319562BD10B562BDB1BC7035B08D1006C
:1006A000DB195C17DB1D5C135B1E5C135F1E722B7A
:1006B000C81B6D2BC81C8712C81C612B87125819C8
:1006C0008716D20B832B5608D200C801D91BC81439
:1006D0005A19C810551AC810832B8712D20B832BB6
:1006E000C803832BC808031987160319832BD20B61
:1006F000832BD71BC8035908D200561ADC17561E85
:10070000DC13DA1FDC135F1F9F2BC91B9A2BC91C3C
:100710000712C91C8E2B071255190716D30BB92BBC
:100720005808D300C901D61BC914D91AC910D81941
:10073000C910B92B0712D30BB92BC903B92B5F1CF6
:10074000AA2BD30BB92B5708D300D61B5D14D81F87
:100750005D10B92BC908031907160319B92BD30B60
:10076000B92BD51AC9035808D300D61B5D14D81F5E
:100770005D10DF1CD52BCA1BD02BCA1C8711CA1CCD
:10078000C42B8711D51B8715D40B08005508D4003E
:10079000CA01D51BCA14561ACA10D619CA100800A5
:1007A0008711D40B0800CA030800CA08031987156B
:1007B00003190800D40B0800D81BCA035608D4003C
:1007C000591ADD14591EDD10DA1FDD100800C001B2
:1007D000DE080319DE035E184014DE1A40144008D8
:1007E000C0015E1C4014DE1E4014C005C00C5E0C2F
:0207F0000800FF
:084000000D000300050005009E
:02400E00CC33B1
:10420000010003000300030003000200020002009B
:1042100002000000000000000000FF00FF00FF009F
:10422000000000000000000000000000000000008E
:104230000000C000C000C000C000FF00FF00FF0081
:104240000300C300F300CF00FF00C300F300CF0062
:10425000FF00C300F300CF00FF00FF00FF00FF00DE
:10426000FF00FF00FF00FF00FF00FF00FF00FF0056
:10427000FF00FF00FF00FF00FF00FF00FF00FF0046
:10428000FF00FF00FF00FF00FF00FF00FF00FF0036
:10429000FF00FF00FF00FF00FF00FF00FF00FF0026
:1042A000FF00FF00FF00FF00FF00FF00FF00FF0016
:1042B000FF00FF00FF00FF00FF00FF00FF00FF0006
:1042C000FF00FF00FF00FF00FF00FF00FF00FF00F6
:1042D000FF00FF00FF00FF00FF00FF00FF00FF00E6
:1042E000FF00FF00FF00FF00FF00FF00FF00FF00D6
:1042F000FF00FF00FF00FF00FF00FF00FF00AA001B
:00000001FF
